:020000040000FA
:020000000428D2
:08000800FF30A200FF30A3004D
:1000100068208E200030AF200030BB20A501A60153
:10002000A701A801A901AA01AB01A010A901FF30F5
:10003000AC00342024102608290203182028241498
:10004000AE20A4102708290203182728A414AD20E5
:1000500024112808290203182E282415AC20A90AE7
:10006000AC0B1928162833286D202D08AB00201D55
:100070003B28A0143C28A010A01C67282B08A50032
:10008000A010A01C44284D286D202D08A600201D7E
:100090004B28A0144C28A0104128A010A01C5128C7
:1000A0005A286D202D08A700201D5828A014592873
:1000B000A0104E28A010A01C5E2867286D202D08D7
:1000C000A800201D6528A0146628A0105B28080041
:1000D00003309F00CC201F13CF2898187B281819B5
:1000E00085288C1E8B288B138B1B73281A088B1763
:1000F0002015AD0008008B138B1B7B2818121A08E3
:100100001A081A0818168B176D288B138B1B852855
:100110001A088B176D282011080008002311C4202D
:10012000A314C520CC2018139816181218151810EF
:10013000181D9D280C309900A1281819A1280230FB
:100140009900CF2098171813181618111A081A08B2
:100150001A08003099000800B828B828B828A50067
:1001600025080F39A6002408F0392604A400B82871
:10017000240885000800A50025080F39A6002208DC
:10018000F0392604A200C928C628C628230866001C
:100190000800220865000800831603130800831274
:0401A000031308003D
:02400E00103F61
:00000001FF
